:020000040000FA
:100000008316103085000130860073308100831222
:1000100097018F01910191158F0397030F088500B8
:10002000111594018F108F12910A9415940A971349
:10003000971081018C010B118E01D720D720D7207A
:10004000D72001088D008D1F262828280B198E0A1D
:100050000C088E078D0A03198E0A06183728D63029
:100060008D02031837288E080319CF288E039901B3
:100070009A019B019C010E1F452808309900013010
:100080009A0009309B0002309C008E1E4D280430DF
:10009000990709309B0706309C070E1E5528023031
:1000A000990704309B0708309C078E1D5D2801309E
:1000B000990702309B0704309C070E1D6528053008
:1000C0009A0701309B0702309C078E1C6D28023076
:1000D0009A0705309B0706309C070E1C75280130D7
:1000E0009A0702309B0708309C078D1F7B2806303B
:1000F0009B0704309C070D1F812803309B070230AB
:100100009C078D1E872801309B0706309C0708300E
:100110000D1A9C0704308D199C0702300D199C079D
:1001200001308D189C070A301C02031C9A289C0081
:100130009B0A93280A301B02031CA1289B009A0AE1
:100140009A280A301A02031CA8289A00990AA128A2
:100150001908093C031CCF28FF3091008F001908B3
:100160000319B828C42091001A08C4208F00BD28A4
:100170001A080319BD28C4208F001B08C42097004B
:100180001C08C4209400192882078134BB3425340C
:1001900023341B34433441348B340134033445302D
:1001A00091007D308F009700FF309400192885154D
:1001B000110886000510EF2005140F088600851031
:1001C000EF208514170886000511EF200515140887
:1001D00086008511EF2000000000000008006F304D
:1001E00095006400000000000B1DF9280B118C0A1B
:1001F000FC280000000000000000000000000000DB
:1002000000000000000000000000000000000000EE
:1002100000000000000000000000000000000000DE
:1002200000000000000000000000000000000000CE
:1002300000000000000000000000000000000000BE
:080240006400950BF42808008E
:02400E00F53F7C
:00000001FF
